:020000008D2A47
:0800080090000308910083122F
:100010008B1811200B19A92011088300900E100EC7
:1000200009000108B10081012B1C1C28831601174F
:1000300083120310AB0DA728AB1C2B283108113CF1
:10004000031CA22809303102031CA2280310AB0DA7
:10005000AC01B001A7282B1D4C283108083C031C1B
:10006000A22807303102031C38280314AC0D4228A3
:100070003108053C031CA22804303102031CA228CD
:100080000310AC0DB00A3008073C031DA72803106D
:10009000AB0DB001AD01A728AB1DA7283108083C66
:1000A000031CA22807303102031C59280314AD0D8C
:1000B00063283108053C031CA22804303102031CCC
:1000C000A2280310AD0DB00A3008053C031DA72877
:1000D000B303031970282C08AE002D08AF00A22826
:1000E0002C082E02031DA2282D082F02031DA22872
:1000F0001A302D02031DA2286C302C02031D822809
:10010000A0309F281C302C02031D882860309F28B7
:100110002C302C02031D8E2820309F2804302C0206
:10012000031D942840309F2844302C02031D9A2838
:1001300080309F280C302C02031DA0281030B20004
:100140000330B3000130AB008316011383128B1010
:1001500008000B110130AB000330B300831601130C
:10016000831208000A148A148200890083168B13F4
:10017000081555308900AA30890088148B17081E8D
:10018000BF280812831208008312890083160814FE
:100190008312080808009300930BCC2808009400F1
:1001A0005530CB20940BD028080095005530CF2037
:1001B000950BD62808000310961B0314960D080013
:1001C00004309200DB20920BE22808000615603014
:1001D000CB20050806116030CB20080085010F30C8
:1001E0008316850083128614E6200F399600E020DE
:1001F000E6200F39960408009600831685018312C5
:100200008610E02016080F398500E620E020160849
:100210000F398500E620EE20961B0B29080096007A
:100220008316850183128610E02016080F39850099
:100230000516E620E02016080F3985000516E62091
:10024000EE20961B202908000130FC280230FC28F3
:100250000438FC280838FC281038FC282038FC28F2
:100260004038FC288038FC28033092000330850099
:10027000E6201530CF20920B362902308500E6208B
:100280002530CB2008302E210230282104302A21AD
:10029000242996000230960D031801388500153088
:1002A000CB2085100530CB20920B4A290800831201
:1002B0008501831685018312861504309200503023
:1002C0004921083092002108492108309200200875
:1002D000492186110301E72108009A00B220003865
:1002E000031908000F211A0A6D29A500B2201D105C
:1002F000A202031C1D14250AA500B2201D18013EF0
:100300001D10A302031885291D14250AB2201D18EB
:10031000013E1D10A40203189229A201A301A40109
:100320000315080003110800A700A6012808A20071
:100330002908A3002A08A400270875210319A82961
:100340002208A8002308A9002408AA00A60A9C29BC
:100350002608080084000008A300840A0008A400FE
:10036000A201973075212208A8002308A9002408BB
:10037000AA009A309421031DBF292030C029303EA5
:100380000F219D309421303E0F21A0309421303E2A
:100390000F21A3309421303E0F212C300F21A630A5
:1003A0009421303E0F21A9309421303E0F21FB30A3
:1003B0006D21080084000008A800A901AA01A93045
:1003C0009421303E0F212808303E0F21080096006E
:1003D0000310960D200888001608B5202108880013
:1003E0001608013EB520080096000310960D160869
:1003F000C4209B001608013EC4200319032A9C0058
:100400001C0A031D08000C309B0015309C000800DE
:100410002008A2002108A300A401AF307521080024
:100420002008A2002108A300A401AC307521080017
:1004300008220319202A0C30A0001530A100080062
:100440000130991A4030A0070318A10A08001022B1
:10045000031D2F2A9930A0002630A100080001308A
:10046000991A4030A002031CA10308000530D520D2
:100470001F301802031D3F2A013098000800980A17
:1004800008000530D52001301802031D4A2A1F300C
:1004900098000800980308000530D5200310970D38
:1004A000971D3429171434291B08A0001C08A1002B
:1004B00057290A303221F8306D211808E729191B15
:1004C0001822991B272200303221E0306D21403064
:1004D00032212030AA29191B3622991B4122991A50
:1004E00054221808F42100303221E7306D211830F1
:1004F000DA21403032211B30AA29191B3622991BE0
:100500004122991A592200303221F0306D211830E1
:10051000DA21403032212030AA290C3084008001B9
:10052000840A841F8F2A1714013098001030D520B8
:10053000F13086008101640083168501F130860068
:1005400007308100831234210301F421542200304A
:100550003221B2306D2140303221C9306D2150300E
:10056000D520242100303221E0306D21403032216D
:100570002030AA21B0308B00572106080F38FF3AEF
:10058000031DC62A32080319BC2AB2019900191AA0
:100590004C2217185F2297186B2217197D22BC2A4C
:02072E000C3489
:1007300051340734403442340F34A0348634013409
:10074000103427340034E834033400346434003483
:1007500000340A34003400340C3415340034993435
:100760002634003450344C344C3420345634303435
:100770002E34313420342834633429343034343442
:100780002F343134393439343934203462347934C3
:10079000003444342E34203446346C3469346534A7
:1007A00067346C342C3420346434653474346934E4
:1007B000403467346D3478342E3464346534003416
:1007C00046347234653471343A342034003452344F
:1007D0006534633461346C346C343A34203400341E
:1007E000533474346F34723465343A342034003402
:1007F0006F346B34003420344D3448347A34003450
:02400E000100AF
:044200000C00150099
:00000001FF
